:020000040800F2
:100000000004022001020008750F0008790F0008A3
:10001000CD0F0008790F0008A10F000803020008A7
:10002000030200080302000803020008C5290008B3
:10003000030200080302000803020008030200088C
:10004000030200080302000803020008030200087C
:100050000302000803020008B13A0008DD3A000874
:10006000093B0008353B0008613B0008030200081B
:10007000030200080302000803020008030200084C
:10008000030200080302000803020008030200083C
:100090000302000803020008030200088D3B000869
:1000A000030200080302000803020008030200081C
:1000B000D538000803020008030200080302000804
:1000C00003020008030200080302000803020008FC
:1000D00003020008030200088111000895110008BE
:1000E000F53B0008030200080302000803020008B1
:1000F00003020008030200080302000803020008CC
:1001000003020008030200080302000803020008BB
:1001100003020008030200080302000803020008AB
:10012000030200080302000803020008030200089B
:10013000030200080302000803020008030200088B
:10014000030200080302000803020008313100081E
:10015000030200080302000803020008030200086B
:10016000030200080302000803020008030200085B
:10017000030200080302000803020008030200084B
:100180000302000803020008A91100080302000886
:10019000030200080302000803020008030200082B
:1001A000030200080302000803020008030200081B
:1001B000030200080302000803020008030200080B
:1001C00003020008030200080302000803020008FB
:1001D00003020008030200080302000803020008EB
:1001E00003020008030200080302000803020008DB
:1001F00003020008030200080302000803020008CB
:1002000002E000F000F8FEE772B6394880F3088893
:10021000384880F3098838484EF60851CEF200017C
:10022000086040F20000CCF200004EF63471CEF2CD
:1002300000010860BFF34F8FBFF36F8F40F20000E3
:10024000C0F2F0004EF68851CEF200010860BFF314
:100250004F8FBFF36F8F4FF00000E1EE100A4EF6A4
:100260003C71CEF200010860062080F31488BFF3D1
:100270006F8F02F0E5FB03F0B5FA4FF055301F49E0
:100280001B4A91423CBF41F8040BFAE71C49194A4A
:1002900091423CBF41F8040BFAE71A491A4A1B4B3A
:1002A0009A423EBF51F8040B42F8040BF8E70020D5
:1002B0001749184A91423CBF41F8040BFAE702F093
:1002C00003FC03F0F9FA144C144DAC4203DA54F871
:1002D000041B8847F9E700F03FF8114C114DAC4280
:1002E00003DA54F8041B8847F9E702F0EBBB00007F
:1002F0000004022000240220000000080000022068
:10030000000402206840000800240220502402203B
:1003100050240220B43D0220000200080002000820
:1003200000020008000200082DE9F04F2DED108AB0
:10033000C1F80CD0D0F80CD0BDEC108ABDE8F08F1D
:10034000002383F311882846A047002001F0C0FF56
:1003500001F0DEFE00DFFEE770B56FF077031F4CA3
:1003600000256FF07F0623701E236570A570E57071
:1003700025716571A571E57125726672A372E572CA
:1003800000F0DEFC20B10E2325726672A372E572C6
:1003900002F0DAFA044602F00FFB0546D0B9104B22
:1003A0009C4219D001339C4241F2883412BF054669
:1003B00000240125002002F0D1FA0DB100F05AF816
:1003C00000F07AFD00F000FC204600F0F3F800F0A9
:1003D00051F8F9E70024EDE70446EBE7502402204A
:1003E000010007B008B500F06DFBA0F120035842F2
:1003F000584108BD054B07B51B88022101A8ADF87F
:10040000043000F0CBFB03B05DF804FBDC3C0008DB
:1004100010B5202383F311881248C3680BB101F093
:10042000DDFF0023104A4FF47A710E4801F09AFF65
:10043000002383F311880D4C236813B12368013B1B
:100440002360636813B16368013B6360084B1B78EA
:1004500033B9636823B9022000F09EFC3223636045
:1004600010BD00BF5C240220110400087825022082
:1004700070240220454B46492DE9F04153F8042FE2
:10048000013201D1BDE8F0818B42F7D1414C424BA2
:1004900022689A4278D9414B9B6803F1006303F5C7
:1004A000C0339A4270D2002000F0AAFB02203C4BDD
:1004B000187000F067FC3B4B1A6C00221A64196E2E
:1004C0001A66196E596C5A64596E5A66596E596992
:1004D00041F080015961596921F0800159615969E0
:1004E000196941F000511961196921F00051196130
:1004F0001B6972B62C4B2D490B601D682468BFF335
:100500004F8FBFF36F8F2A4BC3F88420BFF34F8FF9
:100510005A6922F480325A61BFF34F8FD3F880209A
:1005200043F6E07EC2F3C906C2F34E32B70752016A
:1005300002EA0E0838463146013948EA000C00F15B
:100540004040B1F1FF3FC3F874C2F5D1203A12F137
:10055000200FEDD1BFF34F8FBFF36F8FBFF34F8FDE
:10056000BFF36F8F5A6922F400325A610022C3F838
:100570005022BFF34F8FBFF36F8F202383F3118877
:10058000AD4685F308882047BDE8F081FC7F01086F
:100590001C80010804800108FF7F0108502402200C
:1005A00070240220003802400080010808ED00E0BD
:1005B00000ED00E02DE9F04F99B0B34C2022FF216F
:1005C000019010A8A66800F019FCB04AA346137861
:1005D000A3B90121AE481170C360202383F31188B1
:1005E000C3680BB101F0FAFE0023AA4A4FF47A71F6
:1005F000A74801F0B7FE002383F31188019B13B1D4
:10060000A54B019A1A600023A44AA349019F994669
:100610001C461D46984613704B600292012000F064
:10062000B1FB002F00F012829B4B1B68002B40F0A7
:100630000D8219B0BDE8F08F0220FFF7D3FE00282D
:1006400040F0FB81019BB9F1000F08BF1F46944B9E
:100650001B8802210BA8ADF82C3000F09FFADDE7D3
:100660004FF47A7000F02EFA031E0393EADB0220A7
:10067000FFF7B8FE82460028E4D0039B581E0428EA
:1006800000F2DD81DFE800F0030E1114170018A856
:100690000523042140F8343D00F080FA54464FF021
:1006A000000856E004217848F6E704217D48F3E786
:1006B00004217D48F0E71C242046043400F0A2FA0F
:1006C00004210B900BA800F069FA2C2CF4D1E5E77B
:1006D000002DB7D0002CB5D00220FFF783FE0546D1
:1006E000002800F0AF8101206C4C00F089FA4FF037
:1006F00000090220207000F045FB5FFA89FA50469D
:1007000000F08EFA074658B1504609F1010900F091
:1007100097FA0028F1D12C46A9460027634B97E7AA
:1007200001233E460220237000F022FBDBF8083054
:100730009E4206D2304600F065FA0130EBD1043615
:10074000F4E70026029BA9462C461E703746524B02
:100750005E6000F0A7FB15B1002C18BF0027FFF763
:1007600049FE5BE7002D3FF46DAF002C3FF46AAF0C
:100770000220029B187000F005FB322000F0A2F965
:10078000B0F1000AC0F25E811AF0030540F05A8110
:1007900006EB0A03DBF80820934200F25381BAF516
:1007A000807F00F24F8155450DDA4FF47A7000F0EA
:1007B00089F90490049B002BC0F24481049B3C4ABD
:1007C000AB540135EFE7C820FFF70CFE05460028C3
:1007D00000F038811F2E11D8C6F1200410AB26F08E
:1007E000030033495445184428BF5446224600F0BC
:1007F000DDFA2246FF212E4800F000FB4FEAAA0A4C
:100800002B4930465FFA8AF200F000FB04460028CC
:1008100000F01A8106EB8A0605469AE70220FFF7E8
:10082000E1FD00283FF40EAF00F030FA00283FF45D
:1008300009AF4FF0000A5346DBF8082092451CD25E
:10084000BAF11F0F12D8109A01320FD02AF003020A
:1008500018A90A4452F8202C0B92184604220BA91E
:100860000AF1040A00F0C6FB0346E5E7504603938D
:1008700000F0C8F9039B0B90EFE718A8042140F89B
:100880004C3D00F08BF964E75024022074250220CF
:100890005C24022011040008782502207024022024
:1008A000DE3C00085424022058240220E03C0008CA
:1008B0007424022018A80023642140F8343D00F07D
:1008C00039F900287FF4BEAE0220FFF78BFD002827
:1008D0003FF4B8AE0B9800F0C5F918AB43F8480DDB
:1008E00004211846CDE718A80023642140F8343DC0
:1008F00000F020F900287FF4A5AE0220FFF772FD7A
:1009000000283FF49FAE0B9800F0BAF918AB43F8FB
:10091000440DE5E70220FFF765FD00283FF492AEA5
:1009200000F0C4F918AB43F8400DD9E70220FFF7F7
:1009300059FD00283FF486AE0BA9142000F0BCF945
:10094000824618A8042140F83CAD00F027F9514632
:100950000BA896E7322000F0B5F8B0F1000AFFF6D8
:1009600071AE1AF0030F7FF46DAE0AEB0803DBF8EB
:10097000082093423FF666AE0220FFF733FD0028C1
:100980003FF460AE2AF0030AC244D0453FF4E1AE22
:10099000404608F1040800F035F904210A900AA83D
:1009A00000F0FCF8F1E74FF47A70FFF71BFD002828
:1009B0003FF448AE00F06AF900283FF4AFAE109B58
:1009C00001330CD0082210A9002000F01FFA0028E3
:1009D0003FF4A4AE2022FF2110A800F00FFAFFF789
:1009E00009FD374801F07AFC23E6002D3FF42AAEDA
:1009F000002C3FF427AE18A80023642140F8343DB2
:100A000000F098F8824600287FF41CAE0220FFF721
:100A1000E9FC00283FF416AE0390FFF7EBFC41F22F
:100A20008830574601F05AFC0B9800F083FA00F02A
:100A300039FA039B1C461D46F0E5054689E64FF052
:100A40000008FFE52546FDE52C4667E6002000F09E
:100A500039F80490049B002BFFF6E3AD012000F071
:100A600087F9049B213B122B3FF6D8AD01A252F827
:100A700023F000BF3906000861060008D10600080F
:100A80001D0600081D0600081D0600086507000871
:100A9000550900081D080008B5080008E708000807
:100AA000150900081D0600082D0900081D0600088C
:100AB000A7090008530700081D060008EB090008F5
:100AC000A08601002DE9F3474FF47A75002402AEA9
:100AD000154F4543DFF8588006F8014D97F900306F
:100AE0005FFA84F95A1C01D0A34212D158F82400AD
:100AF000012231460368D3F820A02B46D0470128B5
:100B000007D10A4B9DF8070083F8009002B0BDE8BA
:100B1000F0870134042CE1D14FF4FA7001F0DEFBD0
:100B20004FF0FF30F2E700BF00240220C42502206E
:100B3000EC3C00082DE9F0474FF47A750646002496
:100B4000134F4D43DFF8508097F900305FFA84F976
:100B50005A1C01D0A34210D158F824000422314677
:100B60000368D3F820A02B46D047042805D1094BB1
:100B7000002083F80090BDE8F0870134042CE3D115
:100B80004FF4FA7001F0AAFB4FF0FF30BDE8F08798
:100B900000240220C4250220EC3C0008074B30B49E
:100BA0001A78074B53F822400A460146236820462C
:100BB000DD69044BAC4630BC604700BFC425022051
:100BC000EC3C0008A0860100F8B50A4C00250A4E4E
:100BD00001F0C0FD094F207030682378834207D9A7
:100BE00001F0B2FD336805440133BD423360F3D9EF
:100BF000F8BD00BFC525022080250220FF7F01002F
:100C000001F054BE00F1006000F5C030006870478C
:100C100000F10060920000F5C03001F0E1BD00007D
:100C2000054B1A68054B1B789B1A834202D9104466
:100C300001F08ABD0020704780250220C5250220D2
:100C400038B5074D04462868204401F085FD28B9D1
:100C500028682044BDE8384001F096BD38BD00BF8B
:100C60008025022010F0030308D1B0F5806F05D86D
:100C700000F10050A0F57120006870470020704717
:100C8000014BC058704700BF20F4F01F064991F88F
:100C9000243033B100230822086A81F82430FFF79A
:100CA000B7BF0120704700BF84250220014B1868A0
:100CB000704700BF002004E01F4BF0B51E681F4BBB
:100CC000C6F30B02360C1F885D68BA4293F90840E0
:100CD00022D09F89BA4221D01F8BBA4206D102226C
:100CE0000C2404FB02335D6893F90840B6F5805F7D
:100CF00016D041F201039E4208BF5A24421E013D14
:100D00000B460A44934215D215F9016F581C4EB197
:100D1000034600F8016CF5E70022E1E70122DFE776
:100D20004124EBE72C2582421D7001D9981C5C7090
:100D3000401AF0BD1846FBE7002004E0042402201E
:100D4000094B5B88B3F5805F09D041F20102934201
:100D500007D10122054B03EB8203D87870470022AC
:100D6000F8E70020704700BF002004E0E43C0008E2
:100D7000022803D14FF48052014B9A61704700BFA3
:100D800000100240022803D14FF08052014B9A61BB
:100D9000704700BF00100240022804D1024A536984
:100DA00083F480535361704700100240002310B554
:100DB000934203D0CC5CC4540133F9E710BD00006A
:100DC00030B5441E14F9010F0B4658B193F9005089
:100DD0000131854206D11AB993F90020801A30BD3D
:100DE000013AEFE7002AF7D1104630BD024603462C
:100DF000981A13F9011B0029FAD1704702440346DF
:100E0000934202D003F8011BFAE770472DE9F0473F
:100E1000234C05468846174694F8243083BB2E465B
:100E2000DFF87C90C7B394F824302BB92022FF213F
:100E300048462662FFF7E2FF94F824004146C0F1DD
:100E4000080504EB8000BD4228BF3D465FFA85FAE5
:100E5000AD00A7EB0A072A462E44FFF7A7FF94F838
:100E60002430A844FFB29A445FFA8AFABAF1080F14
:100E700084F824A0D6D1FFF709FF0028D2D108E0DA
:100E8000266A06EB8306B042CAD0FFF7FFFE0028B1
:100E9000C5D10020BDE8F0870120BDE8F08700BF84
:100EA00084250220024B1A78024B1A70704700BF4B
:100EB000C425022000240220F8B5184C184800F080
:100EC000BBFC2146164800F0E3FC24681548E26E9E
:100ED000154DD2F80438154E43F00203104FC2F8F6
:100EE000043801F0FBF92046114900F0DFFDE26E05
:100EF0000024D2F8043823F00203C2F804384FF477
:100F0000E1332B6056F82400B84202D0294600F0A5
:100F1000F1FB0134042CF5D1F8BD00BF0C3E0008F4
:100F2000C835022040420F00AC250220EC3C0008EE
:100F3000303E000838B50B4B05461A780A4B53F87B
:100F400022400A4B9C420CD0094B00211822184623
:100F5000FFF754FF056001462046BDE8384000F029
:100F6000C9BB38BDC4250220EC3C0008C8350220AE
:100F7000AC250220FEE7000000B59BB0EFF309812D
:100F800068226846FFF712FFEFF30583034B9A6B65
:100F90009A6A9A6A9A6A9A6A9B6AFEE700ED00E08A
:100FA00000B59BB0EFF3098168226846FFF7FEFEAB
:100FB000EFF30583044B9A6B9A6A9A6A9A6A9A6A63
:100FC0009A6A9B6AFEE700BF00ED00E000B59BB0A7
:100FD000EFF3098168226846FFF7E8FEEFF3058327
:100FE000034B5A6B9A6A9A6A9A6A9A6A9B6AFEE7F4
:100FF00000ED00E030B50A44074D91420BD011F8E6
:10100000013B09245840013CF7D040F300032B403A
:1010100083EA5000F7E730BD2083B8ED0023044990
:101020001A465A50C81808334260802BF9D17047CD
:10103000C8250220026843681143016003B11847C4
:1010400070470000024A136843F0C0031360704702
:1010500000440040024A136843F0C0031360704725
:1010600000480040024A136843F0C0031360704711
:10107000007800402DE9F047C66D05463768F469F1
:10108000200734621AD014F0080F0CBF0021802111
:10109000E20748BF41F02001A3074FF0200348BFFB
:1010A00041F04001600748BF41F4807183F311882B
:1010B000281DFFF7BFFF002383F31188E2050AD53F
:1010C000202383F311884FF40071281DFFF7B2FF2E
:1010D000002383F311884FF020094FF0000A14F029
:1010E000200831D13B0616D54FF0200905F1380A0A
:1010F000200610D589F31188504600F06FFA0028B9
:101100002FDA0821281DFFF795FF27F080033360B1
:10111000002383F3118879060DD562060BD52023B1
:1011200083F31188EA6C2B6D9A4201D12B6CEBB9D9
:10113000002383F31188E30620D5AA6E1369EBB16F
:101140005069BDE8F047184789F31188736A28464B
:1011500095F86410194000F0DBFA8AF31188F469FD
:10116000BDE7B06288F31188F469C1E727F0400752
:101170001021281DFFF75EFF3760D9E7BDE8F08733
:1011800008B50348FFF776FFBDE8084001F02ABC28
:101190004826022008B50348FFF76CFFBDE8084069
:1011A00001F020BCB426022008B50348FFF762FF17
:1011B000BDE8084001F016BC2027022037B52D4CB1
:1011C0002D4D204600F08AFA009404F1140000230B
:1011D0004FF40072294900F04BF94FF4007200946B
:1011E00004F13800264B274900F0C4F9264B256648
:1011F0000B21E3652620254C00F0C4F8204600F0C2
:101200006DFA009404F1140000234FF40072204999
:1012100000F02EF94FF40072009404F138001D4BD9
:101220001D4900F0A7F91D4B25660B21E36527201A
:101230001B4C00F0A7F8204600F050FA04F114000F
:10124000009400234FF40072164900F011F904F1E4
:10125000380000944FF40072134B144900F08AF9DF
:10126000134B0B215220E365256603B0BDE83040E7
:1012700000F088B84826022080F937038C27022026
:10128000451000088C2D022000440040B4260220A6
:101290008C290220551000088C2F022000480040A5
:1012A000202702208C2B0220651000088C310220A0
:1012B000007800402E4B002908BF1946037C012B03
:1012C000816630B50CD12B4B984235D12A4B1A6C24
:1012D00042F400321A641A6E42F400321A661B6E2F
:1012E0000A68036EC46D03EB5203B3FBF2F34A6862
:1012F000150442BF23F0070503F0070343EA450343
:10130000E3608B6843F040036360CB68510543F0B2
:101310000103A36042F4967343F0010323604FF08E
:10132000FF33236205D512F010221DD0B2F1805F89
:101330001CD080F8643030BD104B984208D10E4B61
:101340001A6C42F480221A641A6E42F48022C5E7B5
:101350000B4B9842C4D1084B1A6C42F080421A647D
:101360001A6E42F08042B9E77F23E2E73F23E0E7CD
:10137000283D00084826022000380240B4260220FA
:101380002027022000F1604300F01F0209014009FC
:1013900003F56143C9B2800083F80013012300F113
:1013A0006040934000F56140C0F8803103607047B1
:1013B000F8B51546826804460B46AA4200D28568F5
:1013C000A1692669761AB54207D218462A46FFF760
:1013D000EDFCA3692B44A3610DE011D9AF1B32468C
:1013E0001846FFF7E3FC3A46E1683044FFF7DEFCBD
:1013F000E2683A44A261A36828465B1BA360F8BD7B
:1014000018462A46FFF7D2FCE368E4E78368934274
:101410002DE9F04104460F46154600D28568606903
:101420002669361AB54207D22A463946FFF7BEFC6E
:1014300063692B4463610EE013D9A5EB06083246BD
:101440003946FFF7B3FC4246B919E068FFF7AEFC36
:10145000E26842446261A36828465B1BA360BDE862
:10146000F0812A463946FFF7A1FCE368E2E7000075
:1014700010B50A440024C361029B00604060846090
:10148000C160816141610261036210BD08B582697A
:101490004369934201D1826882B9826801328260D5
:1014A0005A1C42611970426903699A4201D3C368A8
:1014B0004361002100F02EFF002008BD4FF0FF30F7
:1014C00008BD000070B5202304460E4683F3118842
:1014D000A568A5B1A368A269013BA360531CA361E1
:1014E00015782269934224BFE368A361E3690BB1D5
:1014F00020469847002383F31188284670BD314663
:10150000204600F0F7FE0028E2DA85F3118870BD6E
:101510002DE9F74F05460F4690469A46D0F81C90A5
:10152000202686F311884FF0000B144664B1224642
:1015300039462846FFF73CFF034668B9514628461E
:1015400000F0D8FE0028F1D0002383F31188A8EB27
:10155000040003B0BDE8F08FB9F1000F03D0019093
:101560002846C847019B8BF31188E41A1F4486F371
:101570001188DBE7C160816141611144C361009B57
:10158000006040608260016103627047F8B5044604
:101590000E461746202383F31188A568A5B1A368DA
:1015A000013BA36063695A1C62611E702369626912
:1015B0009A4224BFE3686361E3690BB12046984710
:1015C000002080F31188F8BD3946204600F092FED5
:1015D0000028E2DA85F31188F8BD000083694269CA
:1015E0009A4210B501D182687AB98268013282606C
:1015F0005A1C82611C7803699A4201D3C3688361D3
:10160000002100F087FE204610BD4FF0FF3010BDD6
:101610002DE9F74F05460F4690469A46D0F81C90A4
:10162000202686F311884FF0000B144664B1224641
:1016300039462846FFF7EAFE034668B95146284670
:1016400000F058FE0028F1D0002383F31188A8EBA6
:10165000040003B0BDE8F08FB9F1000F03D0019092
:101660002846C847019B8BF31188E41A1F4486F370
:101670001188DBE7026843681143016003B1184732
:10168000704700001430FFF743BF00004FF0FF33F6
:101690001430FFF73DBF00003830FFF7B9BF00003E
:1016A0004FF0FF333830FFF7B3BF00001430FFF7BF
:1016B00009BF00004FF0FF311430FFF703BF0000F7
:1016C0003830FFF763BF00004FF0FF323830FFF7CC
:1016D0005DBF000000207047FFF770BD044B036042
:1016E000002343608360C36001230374704700BF1D
:1016F000403D000810B52023044683F31188FFF70E
:10170000D9FD02232374002383F3118810BD000048
:1017100038B5C36904460D461BB904210844FFF7D8
:10172000A9FF294604F11400FFF7B0FE002806DAED
:10173000201D4FF48061BDE83840FFF79BBF38BDE6
:10174000026843681143016003B118477047000005
:1017500013B5446BD4F894341A681178042915D160
:10176000217C022912D11979012312898B4013425D
:101770000CD101A904F14C0001F03CFFD4F89444D1
:101780000246019B2179206800F0E0F902B010BD0B
:10179000143001F0BFBE00004FF0FF33143001F0F1
:1017A000B9BE00004C3001F091BF00004FF0FF3394
:1017B0004C3001F08BBF0000143001F08DBE0000F2
:1017C0004FF0FF31143001F087BE00004C3001F0C3
:1017D0005DBF00004FF0FF324C3001F057BF0000FA
:1017E000D0F8942438B5136805461978042901D037
:1017F000012038BD017C0229FAD1127901205C89CF
:1018000090400440F4D105F1140001F01FFE02469F
:101810000028EDD0D5F894544FF480732868697986
:1018200000F082F9204638BD406BFFF7D9BF0000B9
:1018300000207047704700007FB5124B012502263B
:10184000044603600023057400F1840243602946C6
:101850008360C3600C4B0290143001934FF480738B
:10186000009601F0CFFD094B04F523722946019340
:1018700004F14C004FF480730294009601F096FE40
:1018800004B070BD683D0008291800085117000811
:101890000B68202282F311880A7903EB820210621E
:1018A0004A790D3243F822008A7912B103EB8203A0
:1018B00018620223C0F894140374002383F3118880
:1018C0007047000038B5037F044613B190F85430D8
:1018D000ABB90125201D0221FFF732FF04F11400EE
:1018E00025776FF0010100F021FD84F8545004F1D8
:1018F0004C006FF00101BDE8384000F017BD38BD65
:1019000010B5012104460430FFF71AFF00232377A6
:1019100084F8543010BD000038B50446002514305A
:1019200001F088FD04F14C00257701F057FE201DE1
:1019300084F854500121FFF703FF2046BDE83840EA
:10194000FFF74EBF90F85C3003F06003202B19D1F5
:1019500090F85D20212A0AD0222A4FF000030ED0F1
:10196000202A0FD1084A02650722426504E0064B8F
:1019700003650723436500238365012070470365E2
:101980004365F9E70020704728240220D0F89434FA
:1019900037B51A680446117804291AD1017C022946
:1019A00017D11979012312898B40134211D100F10B
:1019B0004C05284601F0D2FE58B101A9284601F095
:1019C00019FED4F894440246019B2179206800F066
:1019D000BDF803B030BD000000EB8103F7B51C6A11
:1019E00005460E46F4B1202383F3118805EB8607E4
:1019F000201D08214C34FFF7A3FEFB685B691B68C0
:101A000013B1204601F004FE01A9204601F0F2FDC9
:101A1000024648B1019B3146284600F097F8002362
:101A200083F3118803B0F0BDFB685A691268002A7D
:101A3000F5D01B8A013B1340F1D105F15C02EAE7C6
:101A40000D3138B550F82140DCB1202383F31188E3
:101A5000D4F894241368527903EB8203DB689B6902
:101A60005D6845B104216018FFF76AFE294604F15C
:101A7000140001F0F5FC2046FFF7B2FE002383F3CB
:101A8000118838BD7047000001F0A4B8012300F1AF
:101A9000240200F1380103700023436042F8043B44
:101AA0008A421361FAD103814381704738B50446F5
:101AB000202383F3118800254160C56005614561DD
:101AC0008561C561056201F095F80223237085F3F5
:101AD000118838BD70B500EB8103054650690E468C
:101AE0001446DA6018B110220021FFF787F9A069C7
:101AF00018B110220021FFF781F931462846BDE8D0
:101B0000704001F041B90000028902F00102028137
:101B1000428902F001024281002202614261826137
:101B2000C261026201F0C4B9F0B4012500EB810486
:101B300047898D40E4683D43A469458123600023C3
:101B4000A2606360F0BC01F0DFB90000F0B40125D1
:101B500000EB810407898D40E4683D436469058199
:101B600023600023A2606360F0BC01F059BA00005A
:101B700070B50223002504460370A0F8645080F875
:101B8000665080F8675005814581C56005614561F3
:101B90008561C561056280F84C5001F091F8636879
:101BA0001B6823B129462046BDE87040184770BD28
:101BB0000278436880F8682005221B6802700BB128
:101BC0000421184770470000436890F868201B689C
:101BD00002700BB1052118477047000090F84C3097
:101BE00070B5044613B1002380F84C3004F15C0258
:101BF000204601F07FF963689B6863BB94F85C50F2
:101C000015F0600615D194F85D3005F07F0545EAC2
:101C1000032540F202339D4200F00E815BD8022D75
:101C200000F0DC803FD8002D00F08780012D00F00F
:101C3000CF800021204601F0C7FB0021204601F0A3
:101C4000B9FB63681B6813B1062120469847062339
:101C500084F84C3070BD204698470028CED094F8C8
:101C6000632094F8623043EA0223626D934238BFE6
:101C7000636594F95C30656D002B4FF0200380F2B2
:101C8000FD80002D00F0EC80092284F84C2083F3C5
:101C900011880021636D226D2046FFF757FF002356
:101CA00083F3118870BDB5F5817F00F0B180B5F583
:101CB000407F49D0B5F5807FBBD194F85E30012BD1
:101CC000B7D1B4F8643023F00203A4F86430266579
:101CD0006665A665C3E740F201639D421ED8B5F56F
:101CE000C06F3BD2B5F5A06FA3D1B4F85C30B3F5AB
:101CF000A06F0ED194F85E30204684F8663001F073
:101D000037F863681B6813B1012120469847032305
:101D10002370002323656365A365A0E7B5F5106F05
:101D200032D040F602439D4252D0B5F5006F80D1CB
:101D300004F167032365012324E004F16403A5652E
:101D40002365022363658AE794F85E30012B7FF4F4
:101D500070AFB4F8643043F00203B6E794F8612042
:101D60002046616894F860304D6843EA022394F895
:101D70005F1094F85E20A84700283FF45AAF4368EC
:101D8000236503686365A4E72378042B10D120231F
:101D900083F311882046FFF7B7FE86F31188636846
:101DA000032184F867601B6821700BB120469847B7
:101DB00094F85E30002BACD084F867300423237095
:101DC00063681B68002BA4D0022120469847A0E737
:101DD000374B23650223636500239DE794F8601069
:101DE000204611F0800F01F00F010ED001F074F8C1
:101DF000012806D002287FF41CAF2E4B60652365B6
:101E000067E72D4B6565236563E701F057F8EFE75A
:101E100094F85E30002B7FF40CAF94F8603013F030
:101E20000F013FF476AF1A06204602D501F0E0FA22
:101E30006FE701F0D3FA6CE794F85E30002B7FF483
:101E4000F8AE94F8603013F00F013FF462AF1B0658
:101E5000204602D501F0B8FA5BE701F0ABFA58E78B
:101E6000142284F84C2083F311882B462A462946F5
:101E70002046FFF759FE85F3118870BD5DB115222C
:101E800084F84C2083F311880021636D226D204675
:101E9000FFF74AFE03E70B2284F84C2083F31188F6
:101EA0002B462A4629462046FFF750FEE3E700BFAF
:101EB000983D0008903D0008943D000838B590F822
:101EC0004C300446152B29D8DFE803F03E2828289B
:101ED00028283E28280B2939282828282828282877
:101EE0003E3E90F8631090F86220436D42EA012272
:101EF0009A4214D9C268128AB3FBF2F502FB153577
:101F00006DB9202383F311882B462A462946FFF713
:101F10001DFE85F311880A2384F84C3038BD142344
:101F200084F84C30202383F31188002320461A467E
:101F30001946FFF7F9FD002383F3118838BD836D3F
:101F400003B198470023E7E7002101F03DFA0021A3
:101F5000204601F02FFA63681B6813B10621204662
:101F600098470623D8E7000090F84C20152A38B58A
:101F7000044622D80123934040F6416213421DD10A
:101F800013F480150FD19B0217D50B2380F84C302A
:101F9000202383F311882B462A462946FFF7D6FDD6
:101FA00085F3118838BDC3689B695B682BB9836D65
:101FB00003B19847002384F84C3038BD002101F06C
:101FC00003FA0021204601F0F5F963681B6813B19C
:101FD0000621204698470623EDE70000024B002229
:101FE0001B605B609A6070478C330220002382681C
:101FF0000374054B1B6899689142FBD25A680360D1
:1020000042601060586070478C33022008B520236E
:1020100083F31188037C032B05D0042B0DD02BB93F
:1020200083F3118808BD436900221A604FF0FF3323
:102030004361FFF7DBFF0023F2E790E80C001A6032
:1020400002685360F2E70000002382680374054BC6
:102050001B6899689142FBD85A680360426010601F
:10206000586070478C330220054B19690874186852
:10207000026853601A60186101230374FEF754B9B3
:102080008C3302204B1C30B5054687B00A4C10D06B
:10209000236901A8094A00F065F92846FFF7E4FF23
:1020A000049B13B101A800F099F92369586907B09E
:1020B00030BDFFF7D9FFF8E78C3302200D20000870
:1020C00038B50C4D044641612B6981689A6891428C
:1020D00003D8BDE83840FFF789BF1846FFF786FFF1
:1020E00001232C61014623742046BDE83840FEF7E9
:1020F0001BB900BF8C330220044B1A681B6990681F
:102100009B68984294BF0020012070478C330220C6
:1021100010B5084C236820691A68546022600122B7
:1021200023611A74FFF790FF01462069BDE8104053
:10213000FEF7FAB88C330220FEE7000010B5194C08
:10214000FFF74CFF00F000F980221749204600F00D
:1021500085F8012344F8180C0374144B144AD96809
:1021600021F4E0610904090C0A431249DA60CA68E3
:1021700042F08072CA60104A1049C2F8B01F11685C
:1021800041F0010111601022DA77202283F8222029
:10219000002383F3118862B60948BDE8104000F0BF
:1021A0007FB800BFB43302209C3D000800ED00E082
:1021B0000003FA05F0ED00E0001000E055CEACC5DC
:1021C000A43D00082DE9F84F1E4C4FF0000865694A
:1021D00004F11407C1464FF08043266AAA685B6A7F
:1021E0009E1B96421CD34FF0200AAA68236AD5F89A
:1021F0000CB0B61A134423622B68BB425F60636164
:10220000C5F80C8001D101F0D3FA89F3118828694F
:10221000D8478AF311886569AB689E42E5D2DAE750
:102220006269BA420CD0916823628E1B9660A868DE
:1022300002282CBF1818981CBDE8F84F01F0BEBA50
:10224000BDE8F88F8C330220034B59685A68521A44
:102250009042FBD8704700BF001000E0826002226D
:1022600002740022427470478368A3F17C0243F831
:102270000C2C026943F83C2C426943F8382C074A7D
:1022800043F81C2CC268A3F1180043F8102C02225A
:1022900003F8082C002203F8072C704741030008BC
:1022A00010B5202383F31188FFF7DEFF00210446D9
:1022B000FFF706FF002383F31188204610BD0000BE
:1022C000024B1B6958610F20FFF7CEBE8C330220F2
:1022D000202383F31188FFF7F3BF000008B5014600
:1022E000202383F311880820FFF7CCFE002383F31B
:1022F000118808BD49B1064B42681B6918605A60D5
:10230000136043600420FFF7BDBE4FF0FF307047FD
:102310008C3302200368984206D01A68026050602D
:1023200018465961FFF762BE7047000038B5044691
:102330000D462068844200D138BD036823605C608C
:102340004561FFF753FEF4E7054B03F114025A61B0
:102350009A614FF0FF32DA6100221A62704700BFC3
:102360008C330220F8B503614FF08043C26002292C
:102370005C6A0646184B38BF02211A461F4652F8BF
:10238000145F95420AD1586198611C6205604560EE
:1023900081600819BDE8F84001F002BA186AAB681C
:1023A000241A0C1902D3E41A2D6804E09C4202D2CC
:1023B000204401F003FAAB689C42F4D86B683560A6
:1023C00073601E604FF0FF336E60B460A968091B34
:1023D000A960FB61F8BD00BF8C33022010B41B4C18
:1023E000234653F8141F814210D0416802680A60E6
:1023F000026851609A424FF00001C16003D09368B7
:1024000081680B4493605DF8044B70470A680020B4
:102410009A4262615360C86003D15DF8044B01F0D9
:10242000C7B9936888680344206A93604FF080427C
:10243000526A121A9342E6D9991A5DF8044B01299F
:1024400098BF931C184401F0B9B900BF8C33022027
:1024500000207047FEE70000704700004FF0FF309B
:1024600070470000022906D0032906D0012906483A
:1024700018BF0020704705487047032A9ABF0448D8
:1024800000EBC200002070478C3E0008403E000870
:102490003024022070B59AB006460846144601ADB5
:1024A000294600F095F82846FEF7A0FCC0B2431C70
:1024B0005B0086E8180023700323023404F8013C13
:1024C00000231946DAB20234904201D81AB070BD26
:1024D000EA5C013304F8011C04F8022CF2E7000066
:1024E00008B5202383F311880348FFF74FFA002330
:1024F00083F3118808BD00BFC835022010B504461B
:10250000052916D8DFE801F016150316161D20233D
:1025100083F311880E4A0121FFF7DCFA20460D4AA9
:102520000221FFF7D7FA0C48FFF7F6F9002383F3EF
:10253000118810BD202383F311880748FFF7C2F9E3
:10254000F4E7202383F311880348FFF7D9F9EDE777
:10255000C43D0008E83D0008C835022038B50C4DE0
:102560000C4C2A460C4904F10800FFF793FF05F1D3
:10257000CA0204F110000949FFF78CFF05F5CA7281
:1025800004F118000649BDE83840FFF783BF00BFDB
:10259000903A022030240220143E0008183E000821
:1025A000243E000870B5044608460D46FEF71EFCA2
:1025B000C6B22046013403780BB9184670BD3246C6
:1025C0002946FEF7FDFB0028F3D1012070BD000075
:1025D0002DE9F84F05460C46FEF708FC2C49C6B21B
:1025E0002846FFF7DFFF08B10336F6B2294928462F
:1025F000FFF7D8FF08B11036F6B2632E0DD8DFF81A
:102600009080DFF89090244FDFF894A0DFF894B02A
:102610002E7846B92670BDE8F88F29462046BDE8D9
:10262000F84F01F053BB252E2ED1072241462846F4
:10263000FEF7C6FB70B9DBF8003007350A3444F802
:102640000A3CDBF8043044F8063CBBF8083024F8B8
:10265000023CDDE7082249462846FEF7B1FB98B95F
:10266000A21C0E4B13F8011F023209095345C95D24
:1026700002F8041C197801F00F01C95D02F8031C6F
:10268000F0D118340835C3E7267001350134BFE7AF
:10269000AC3E0008243E0008BF3E00081FF4F01FB7
:1026A0002BF4F01FB43E0008BFF34F8F024AD368EB
:1026B000DB03FCD4704700BF003C024008B5074B69
:1026C0001B7853B9FFF7F0FF054B1A69002A04DAAB
:1026D000044A5A6002F188325A6008BDEE3C02207A
:1026E000003C02402301674508B5054B1B7833B910
:1026F000FFF7DAFF034A136943F00043136108BD93
:10270000EE3C0220003C02400B2870B513D80B4A67
:102710000B4C137863B94FF000610A4E44F8231054
:1027200056F8235001330C2B2944F7D101231370A1
:1027300054F8200070BD002070BD00BF203D022075
:10274000F03C0220D03E0008014B53F820007047B7
:10275000D03E00080C2070470B2810B5044601D964
:10276000002010BDFFF7D0FF064B53F8243018446B
:10277000C21A0BB9012010BD12680132F0D1043B1E
:10278000F6E700BFD03E00080B2810B5044621D85C
:10279000FFF78AFFFFF792FF0F4AF323D360C300CE
:1027A000DBB243F4007343F002031361136943F493
:1027B00080331361FFF778FFFFF7A6FF074B53F84D
:1027C000241000F0DBF8FFF78FFF2046BDE8104033
:1027D000FFF7C2BF002010BD003C0240D03E000801
:1027E0002DE9F84312F0010315463FD18218B2F1EA
:1027F000026F3BD22B4B1B6813F0010336D0FFF75F
:102800005DFF294CF32340F20127E360FFF74CFF03
:10281000032D01D9830712D00F46401A224C40F2F3
:102820000118EB1BC6190B44012B236924D823F094
:1028300001032361FFF758FF0120BDE8F8832369F6
:1028400023F44073236123693B43236151F8046BF4
:102850000660BFF34F8FFFF727FF03689E4208D043
:10286000236923F001032361FFF73EFF0020BDE849
:10287000F883043D0430CBE723F44073B946236169
:10288000236943EA0803236137F8023B3380BFF32F
:102890004F8FFFF709FF3688B6B2B9F80030B34260
:1028A000BFD0DDE700380240003C0240084908B5CF
:1028B0000B7828B153B9FFF701FF01230B7008BD56
:1028C00023B10870BDE80840FFF70EBF08BD00BF88
:1028D000EE3C022002440439064BD2B210B59042BD
:1028E00000D110BD441C00B253F8200041F8040F81
:1028F000E0B2F4E750280040104B30B51C6F2404C0
:1029000007D41C6F44F400741C671C6F44F400442B
:102910001C670B4C024404392368D2B243F4807321
:102920002360084B904200D130BD441C51F8045F35
:1029300000B243F82050E0B2F4E700BF0038024094
:10294000007000405028004007B5012201A9002076
:10295000FFF7C0FF019803B05DF804FB13B5044610
:10296000FFF7F2FFA04206D002A90122002041F8A1
:10297000044DFFF7C1FF02B010BD00000144BFF3DA
:102980004F8F064B884204D3BFF34F8FBFF36F8F37
:102990007047C3F85C022030F4E700BF00ED00E0B0
:1029A000034B1B689B0042BF0122024B1A70704709
:1029B00074380240213D0220014B1878704700BF57
:1029C000213D0220064A536823F001035360EFF3D0
:1029D0000983683383F30988002383F311887047E0
:1029E00030EF00E010B5202383F31188104B5B68B3
:1029F00013F4006318D0F1EE103AEFF309844FF0AE
:102A0000807344F84C3C0B4BDB6844F8083CA4F161
:102A1000680383F30988FFF76FFB18B1064B44F88E
:102A2000503C10BD054BFAE783F3118810BD00BF81
:102A300000ED00E030EF00E051030008540300080F
:102A4000F0B5BFF34F8FBFF36F8F1D4B0021C3F85D
:102A50005012BFF34F8FBFF36F8F5A6942F40032A9
:102A60005A61BFF34F8FBFF36F8FC3F88410BFF36A
:102A70004F8FD3F8802043F6E076C2F3C904C2F347
:102A80004E32A507520102EA060E284621464EEABA
:102A90000007013900F14040C3F860724F1CF6D1C5
:102AA000203A12F1200FEED1BFF34F8F5A6942F452
:102AB00080325A61BFF34F8FBFF36F8FF0BD00BFFD
:102AC00000ED00E0FEE70000084A094B09498B428F
:102AD00004D3094A0021934205D3704752F8040FEA
:102AE00043F8040BF3E743F8041BF4E7B440000891
:102AF000B43D0220B43D0220B43D0220036F002209
:102B000030B51146C46E9D684FF0FF3004EB4213A0
:102B100001329542C3F80019C3F81019C3F8080927
:102B2000C3F8001BC3F8101BC3F8080BEED24FF01C
:102B30000113C4F81C3830BD890141F02001016146
:102B400003699B06FCD41220FFF77EBB204B03EBEE
:102B500080022DE9F047D2F80CE0461CDD6EDEF86D
:102B6000142005EB0636D2F800C005EB401851687A
:102B700061450BD30123D5F8342803FA00F022EA8B
:102B80000000C5F834081846BDE8F087ACEB010337
:102B9000BEF81040A34228BF2346D8F81849A4B273
:102BA000B3EB840F10D894681F46A4F1040959F8B8
:102BB00004AF042FC6F800A001D9043FF7E71C4476
:102BC0000B4494605360D2E70020BDE8F08700BF5B
:102BD000243D022010B5054C2046FEF757FF4FF06C
:102BE000A043E366024B236710BD00BF243D0220D3
:102BF000243F00080378012B70B5054650D12A4BBD
:102C0000C46E98421BD1294B0E2143205A6B42F0CF
:102C100080025A635A6D42F080025A655A6D5A69B1
:102C200042F080025A615A6922F080025A615B695F
:102C3000FEF7A8FB1E4BE3601E4BC4F800380023D0
:102C4000EE6EC4F8003EC02323604FF40413A36368
:102C50003369002BFCDA01230C203361FFF7F4FA0F
:102C60003369DB07FCD41220FFF7EEFA3369002B3F
:102C7000FCDA00262846A660FFF740FF6B68C4F820
:102C80001068DB68C4F81468C4F81C684BB90A4BB8
:102C9000A3614FF0FF336361A36843F00103A360B6
:102CA00070BD064BF4E700BF243D0220003802400F
:102CB0004014004003002002003C30C0083C30C0FB
:102CC000F8B5C46E054600214FF000662046FFF7B8
:102CD00033FF296F00234FF001128F684FF0FF3050
:102CE000C4F83438C4F81C2804EB431201339F4263
:102CF000C2F80069C2F8006BC2F80809C2F8080BF4
:102D0000F2D20B68EA6E6B67636210231361166977
:102D100016F01006FBD11220FFF796FAD4F800380F
:102D200023F4FE63C4F80038A36943F4402343F05E
:102D30001003A3610923C4F81038C4F814380A4BEF
:102D4000EB604FF0C043C4F8103B084BC4F8003BA5
:102D5000C4F81069C4F800396B6F03F1100243F432
:102D600080136A67A362F8BD003F0008408000102E
:102D7000C26E90F86610D2F8003823F4FE6343EA7E
:102D80000113C2F8003870472DE9F0410EB20D462C
:102D900000EB8608D8F80C100F6807F00303022B2D
:102DA00050D0032B50D03D4A3D4F012B18BF174642
:102DB000C46E4FEA451E002205F1100C04EB0E0311
:102DC000C3F8102B8A69002A40D04A8A05F15803BB
:102DD0003A435B01E2500123D4F81C2803FA0CF3B8
:102DE0001343C4F81C38A64400234A69CEF81039AE
:102DF00005F13F03002A39D00A8A04EB8303898B4B
:102E00009208012988BF4A43416F561841EA02429D
:102E10002946466720465A60FFF78EFED8F80C30E8
:102E20001B8A43EA85531F4305F148035B01E750C2
:102E30000123D4F81C2803FA05F51543C4F81C58DF
:102E4000BDE8F081174FB3E7174FB1E704EB461326
:102E5000D3F8002B22F40042C3F8002B0123D4F84E
:102E60001C2803FA0CF322EA0303BAE704EB8303FA
:102E70000E4A04EB461629465A602046FFF75CFED0
:102E8000D6F80039012223F4004302FA05F5C6F80A
:102E90000039D4F81C3823EA0505CFE7008000107C
:102EA000008004100080081000800C100004000254
:102EB000026F12684267FFF721BE00005831C36EEF
:102EC00049015B5813F4004004D013F4001F14BFF1
:102ED00001200220704700004831C36E49015B5851
:102EE00013F4004004D013F4001F14BF012002208B
:102EF0007047000000EB8101CB68196A0B68136012
:102F00004B6853607047000000EB810330B5DD680B
:102F1000AA691368D36019B9402B84BF402313609A
:102F20006B8A1468C26E1C4402EB4110013C09B26A
:102F3000B4FBF3F46343033323F0030343EAC443D2
:102F400043F0C043C0F8103B2B6803F00303012B90
:102F50000ED1D2F8083802EB411013F4807FD0F87C
:102F6000003B14BF43F0805343F00053C0F8003BD4
:102F700002EB4112D2F8003B43F00443C2F8003B9D
:102F800030BD00002DE9F041244D0446EE6E06EB05
:102F90004013D3F8087B3807C3F8087B0AD5D6F866
:102FA0001438190706D505EB840321462846DB684B
:102FB0005B689847FA072FD5D6F81438DB072BD56E
:102FC00005EB8403D968CCB98B69488A5E68B6FB87
:102FD000F0F200FB12628AB91868DA6890420DD2EA
:102FE000121A83E81400202383F311880B4821462A
:102FF000FFF78AFF84F31188BDE8F081012303FA0B
:1030000004F26B8923EA02036B81CB6823B121466A
:103010000248BDE8F0411847BDE8F081243D022098
:1030200000EB81034A0170B5DD68C36E6C692668E8
:10303000E66056BB1A444FF40020C2F810092A6813
:1030400002F00302012A0AB20ED1D3F8080803EBFA
:10305000421410F4807FD4F8000914BF40F080506F
:1030600040F00050C4F8000903EB4212D2F8000906
:1030700040F00440C2F800090122D3F8340802FAF3
:1030800001F10143C3F8341870BD19B9402E84BF53
:103090004020206020681A442E8A841940F0005095
:1030A000013CB4FBF6F440EAC440C6E7F8B5044678
:1030B0001E48C56E05EB4413D3F80869F107C3F841
:1030C000086917D5D5F81038DA0713D500EB840353
:1030D000D9684B691F68DA68974218D2D21B00275B
:1030E0001A605F60202383F311882146FFF798FF61
:1030F00087F31188330617D50123D5F83428A34068
:10310000134211D02046BDE8F840FFF71FBD012350
:1031100003FA04F2038923EA020303818B68002B7C
:10312000E8D021469847E5E7F8BD00BF243D0220DE
:103130009F482DE9F84FC56E04466E69AB691E4085
:1031400016F4805F6E6105D0FEF712FDBDE8F84F02
:10315000FFF748BC002E12DAD5F8003E9B0705D0D9
:10316000D5F8003E23F00303C5F8003ED5F8043837
:103170008F4823F00103C5F80438FEF725FD370515
:1031800002D58B48FEF714FDB0040CD5D5F80838ED
:1031900013F0060FEB6823F470530CBF43F4105385
:1031A00043F4A053EB60310704D56368DB680BB1CF
:1031B0007F489847F2026FD4B3020CD5D4F86C80E4
:1031C00000274FF00109DFF8E8A1236FF9B29B68EF
:1031D0008B4280F09C80F70619D5E16E0A6AC2F333
:1031E0000A1702F00F0302F4F012B2F5802F00F07C
:1031F000B580B2F5402F0AD104EB830301F580516D
:10320000DB68186A00231A469F4240F09C80330313
:10321000D5F818481DD5E70302D50020FFF7B2FE08
:10322000A50302D50120FFF7ADFE600302D5022001
:10323000FFF7A8FE210302D50320FFF7A3FEE20259
:1032400002D50420FFF79EFEA30202D50520FFF75A
:1032500099FE77037FF57AAFE60702D50020FFF7E6
:1032600025FFA50702D50120FFF720FF600702D543
:103270000220FFF71BFF210702D50320FFF716FFEF
:10328000E20602D50420FFF711FFA3067FF55EAF2B
:103290000520FFF70BFF59E7D4F86C8000274FF0AB
:1032A0000109DFF80CA1236F5FFA87FB9B685B4580
:1032B00082D308EB4B13D3F8002902F44022B2F575
:1032C000802F22D1D3F80029002A1EDAD3F8002952
:1032D00042F09042C3F80029D3F80029002AFBDB12
:1032E0005946E06EFFF728FC228909FA0BF322EA1F
:1032F0000303238104EB8B03DB689B6813B15946FE
:10330000504698475846FFF721FC0137CBE708EBBA
:103310004112D2F8003B03F44023B3F5802F10D1C3
:10332000D2F8003B002B0CDA628909FA01F322EA99
:103330000303638104EB8103DB68DB680BB1504658
:103340009847013741E79C0700D10A68072B03F132
:1033500001039EBF0270120A013055E7023301F5E6
:10336000805104EB8302526890690268D0F808C06B
:103370004068A2EB000E0022104697420AD104EBEF
:10338000830463689B699A683A449A605A68174450
:103390005F603CE712F0030F00D10868964502F128
:1033A000010282BF8CF80000000A0CF1010CE4E776
:1033B000243D0220C36E03EB4111D1F8003B43F4DE
:1033C0000013C1F8003B7047C36E03EB4111D1F805
:1033D000003943F40013C1F800397047C36E03EBA2
:1033E0004111D1F8003B23F40013C1F8003B7047B2
:1033F000C36E03EB4111D1F8003923F40013C1F877
:103400000039704730B50433039C0172002104FB7E
:103410000325C361049B00600363059B4060C1609A
:10342000426102618561046242628162C1624363FA
:1034300030BD00000022416AC260416101616FF04D
:1034400001018262C262FEF771BF00000369426936
:10345000934203D1C2680AB100207047181D70471B
:10346000036919600021C2680132C260C269134455
:1034700082699342036124BF436A0361FEF74ABF36
:1034800038B504460D46E3683BB162690020131D60
:103490001268A3621344E36238BD237A33B9294624
:1034A0002046FEF727FF0028EDDA38BD6FF0010057
:1034B000FBE70000C368C269013BC3604369134472
:1034C00082699342436124BF436A4361002383625C
:1034D000036B03B11847704770B52023044683F38C
:1034E0001188866A3EB9FFF7CBFF054618B186F30F
:1034F0001188284670BDA36AE26A13F8015B934203
:10350000A36202D32046FFF7D5FF002383F311887F
:10351000EFE700002DE9F84F04460E469046994625
:10352000202787F311880025AA46D4F828B0BBF1DC
:10353000000F09D149462046FFF7A2FF20B18BF3C7
:1035400011882846BDE8F88FA16AA8EB050BE36A4D
:103550005B1A9B4528BF9B46BBF1400F1BD93346E6
:1035600001F1400251F8040B914243F8040BF9D1E8
:10357000A36A403640354033A362A26AE36A9A42A6
:1035800002D32046FFF796FF8AF311884545D8D22B
:1035900087F31188C9E730465A46FDF707FCA36A4E
:1035A0005E445D445B44A362E7E7000010B5029C03
:1035B00004330172C36103FB0421002300608362B2
:1035C000C362039B40600363049BC4604261026169
:1035D000816104624262436310BD0000026A6FF0C1
:1035E0000101C260426A4261026100228262C262DB
:1035F000FEF79CBE436902699A4203D1C2680AB1D0
:1036000000207047184650F8043B0B6070470000DC
:10361000C3680021C2690133C360436913448269EE
:103620009342436124BF436A4361FEF773BE0000C7
:1036300038B504460D46E3683BB1236900201A1DE6
:10364000A262E2691344E36238BD237A33B92946A2
:103650002046FEF74FFE0028EDDA38BD6FF001007E
:10366000FBE7000003691960C268013AC260C269E1
:10367000134482699342036124BF436A03610023B8
:103680008362036B03B118477047000070B52023B5
:1036900004460E4683F31188856A35B91146FFF753
:1036A000C7FF10B185F3118870BDA36A1E70A36AAD
:1036B000E26A01339342A36204D3E16920460439EC
:1036C000FFF7D0FF002080F3118870BD2DE9F84F7F
:1036D00004460D4691469A464FF0200888F311881B
:1036E0000026B346A76A4FB951462046FFF7A0FF10
:1036F00020B187F311883046BDE8F88FA06AA9EBA6
:103700000603E76A3F1A9F4228BF1F46402F1BD976
:1037100005F1400355F8042B9D4240F8042BF9D1E4
:10372000A36A40364033A362A26AE36A9A4204D392
:10373000E16920460439FFF795FF8BF311884E4568
:10374000D9D288F31188CDE729463A46FDF72EFBFA
:10375000A36A3D443E443B44A362E5E702694369F2
:103760009A4203D1C3681BB9184670470023FBE790
:10377000836A002BF8D0043B9B1AF5D01360C36812
:10378000013BC360C3691A4483699A42026124BF42
:10379000436A0361002383620123E5E700F0AEB8CA
:1037A0004FF08043002258631A610222DA607047AA
:1037B00000224FF08043DA60704700004FF08043F2
:1037C000586370474B6843608B688360CB68C36005
:1037D0000B6943614B6903628B6943620B68036049
:1037E0007047000008B5274B40F2FF7126481A6960
:1037F0000A431A611A6922F4FF6222F007021A6171
:103800001A691A6B0A431A631A6D0A431A651F4A2A
:103810001B6D1146FFF7D6FF1D4802F11C01FFF793
:10382000D1FF1C4802F13801FFF7CCFF1A4802F122
:103830005401FFF7C7FF194802F17001FFF7C2FFFB
:10384000174802F18C01FFF7BDFF164802F1A801ED
:10385000FFF7B8FF144802F1C401FFF7B3FF1348A4
:1038600002F1E001FFF7AEFF114802F1FC01FFF7A2
:10387000A9FF104802F58C71FFF7A4FFBDE80840CE
:1038800000F09EB80038024000000240303F0008BF
:103890000004024000080240000C024000100240F8
:1038A0000014024000180240001C024000200240A8
:1038B000002402400028024008B500F0F5F9FEF7A8
:1038C0003DFCFFF76DF8BDE80840FEF747BE00007D
:1038D000704700004FF080431A69920710B508D571
:1038E00000241C61202383F31188FEF76BFC84F312
:1038F0001188BDE81040FFF775B80000104B082193
:103900001C201A6C42F001021A641A6E42F0010285
:103910001A660C4A1B6E936843F0010393604FF0E4
:1039200080436B229A624FF0FF32DA6200229A6182
:103930005A63DA605A6001225A611A60FDF722BDAB
:1039400000380240002004E01B4B4FF0FF30002104
:103950001A696FEA42526FEA52521A611A69C2F347
:103960000A021A611A695A6958615A6959615A6991
:103970001A6A62F080521A621A6A02F080521A625F
:103980001A6A5A6A58625A6A59625A6A0B4A106825
:1039900040F480701060186F00F44070B0F5007F44
:1039A00003D04FF4803018671967536823F400730D
:1039B000536000F059B900BF003802400070004069
:1039C000354B4FF44041354A1A64354A11601A6844
:1039D00042F001021A601A689207FCD59A6822F038
:1039E00003029A602C4B19469A6812F00C02FBD124
:1039F000186800F0F90018609A601A6842F4803282
:103A00001A600B689B03FCD54B6F43F001034B67B7
:103A1000214B5A6F9007FCD5224A5A601A6842F02F
:103A200080721A601E4B1A4659684904FCD5196801
:103A300041F4803119605368D803FCD5136843F40E
:103A400000331360164A53689903FCD5124B1A6869
:103A50009201FCD5144A40F207319A6040F20112FB
:103A6000C3F88C200022C3F89020104A11609A6895
:103A700042F002029A60084B9A6802F00C02082A8F
:103A8000FAD15A6C42F480425A645A6E42F480422F
:103A90005A665B6E704700BF003802400004001099
:103AA00000700040186C400900948838003C0240C7
:103AB000084A08B5536911680B4003F001035361CC
:103AC00023B1054A13680BB150689847BDE8084018
:103AD000FEF788BF003C0140C8250220084A08B50F
:103AE000536911680B4003F00203536123B1054A87
:103AF00093680BB1D0689847BDE80840FEF772BFE5
:103B0000003C0140C8250220084A08B553691168E5
:103B10000B4003F00403536123B1054A13690BB151
:103B200050699847BDE80840FEF75CBF003C014083
:103B3000C8250220084A08B5536911680B4003F0F4
:103B40000803536123B1054A93690BB1D0699847C3
:103B5000BDE80840FEF746BF003C0140C8250220F2
:103B6000084A08B5536911680B4003F0100353610C
:103B700023B1054A136A0BB1506A9847BDE8084063
:103B8000FEF730BF003C0140C8250220174B10B59E
:103B90005C691A68144004F478725A61A30604D56B
:103BA000134A936A0BB1D06A9847600604D5104A4D
:103BB000136B0BB1506B9847210604D50C4A936BDD
:103BC0000BB1D06B9847E20504D5094A136C0BB1D1
:103BD000506C9847A30504D5054A936C0BB1D06C83
:103BE0009847BDE81040FEF7FDBE00BF003C014015
:103BF000C82502201A4B10B55C691A68144004F4F9
:103C00007C425A61620504D5164A136D0BB1506DA2
:103C10009847230504D5134A936D0BB1D06D98478F
:103C2000E00404D50F4A136E0BB1506E9847A104FF
:103C300004D50C4A936E0BB1D06E9847620404D53C
:103C4000084A136F0BB1506F9847230404D5054AF7
:103C5000936F0BB1D06F9847BDE81040FEF7C2BE1E
:103C6000003C0140C8250220062108B50846FDF7A2
:103C700089FB06210720FDF785FB06210820FDF7BB
:103C800081FB06210920FDF77DFB06210A20FDF7B7
:103C900079FB06211720FDF775FB06212820BDE8DA
:103CA0000840FDF76FBB000008B5FFF74DFEFDF7BC
:103CB000B5F9FDF711FDFDF7E7FEFDF7BBFDFFF7D9
:103CC00007FEBDE80840FFF769BD0000034611F894
:103CD000012B03F8012B002AF9D17047121012139F
:103CE000121100000010410001105A00C8350220D6
:103CF00048260220B42602202027022053544D33A8
:103D000032463F3F3F3F3F3F0053544D33324637EB
:103D10005B347C355D780053544D333246375B3627
:103D20007C375D7800000000009600000000000075
:103D30000000000000000000000000000000000083
:103D400000000000A11600088D160008C916000822
:103D5000B5160008C1160008AD160008991600082F
:103D600085160008D516000800000000AD170008F1
:103D700099170008D5170008C1170008CD170008CB
:103D8000B9170008A5170008911700083118000896
:103D90000000000001000000000000006D61696E7D
:103DA00000000000BC3D0008D0330220C8350220CE
:103DB00001000000392100080000000069646C6502
:103DC000000000000200000000000000D9190008F7
:103DD000411A000840004000603A0220703A022078
:103DE00002000000000000000300000000000000CE
:103DF000851A00080000000010000000803A022030
:103E0000000000000100000000000000243D02202E
:103E1000010102006D526F0058322E312D373737B5
:103E20002D424C002553455249414C2500000000CD
:103E3000FD2400086524000845190008E124000855
:103E400043000000483E000809024300020100C090
:103E500032090400000102020100052400100105DE
:103E60002401000104240202052406000107058242
:103E7000030800FF09040100020A00000007050111
:103E8000024000000705810240000000120000000F
:103E9000943E00081201100102000040091241572F
:103EA00000020102030100000403090425424F41FE
:103EB000524425006D526F5832312D37373700305C
:103EC0003132333435363738394142434445460080
:103ED00000800000008000000080000000800000E2
:103EE00000000200000004000000040000000400C4
:103EF00000000400000004000000040000000400B2
:103F000000000000DD1B0008BD1E0008691F00083E
:103F1000400040009C3D02209C3D0220010000002A
:103F2000AC3D0220800000004001000005000000C0
:103F30000000802A00000000AAAAAAAA000000002F
:103F4000FFFF00000000000000A00A0000000000C9
:103F500000000000AAAAAAAA00000000FFFF0000BB
:103F600000000000000000001400004000000000FD
:103F7000AAAAAAAA14000040FFFF00000000000047
:103F80000000000080699A0100000000AAAA8AAA25
:103F900040555501FFFF000000707007777000006A
:103FA0000080020100000000AAAAAAAA00400100A5
:103FB000FFFF00000000008008000000000000007B
:103FC00000000000AAAAAAAA00000000FFFF00004B
:103FD00000000000000000000000000000000000E1
:103FE000AAAAAAAA00000000FFFF0000000000002B
:103FF000000000000000000000000000AAAAAAAA19
:1040000000000000FFFF00000000000000000000B2
:104010000000000000000000AAAAAAAA00000000F8
:10402000FFFF000000000000000000000000000092
:104030000000000000000000000000000000000080
:104040000000000000000000000000000000000070
:104050000000000000000000000000000000000060
:104060000000000000000000FF0000000000000051
:10407000FC3C00083F00000049040000093D000826
:104080003F00000051040000173D00083F00000001
:10409000009600000000080004000000A83E000890
:1040A0000000000000000000000000000000000010
:0840B000000000000000000008
:00000001FF
